:020000040800F2
:10A0000080D9002061A10008F9B000083DAD00082A
:10A01000C9B00008D9A200082DBA0008000000004D
:10A0200000000000000000000000000071B80008FF
:10A030002DA900080000000085B60008B1B800088E
:10A04000C1A10008C1A1000801BA000841B500087B
:10A05000A9B50008A9A90008C1A1000889A800089D
:10A06000C1A10008C1A10008C1A10008C1A1000848
:10A07000D1B10008C1A1000829B50008C1A100089C
:10A08000C1A10008C1A10008C1A10008C1A1000828
:10A09000C1A10008C1A10008C1A10008C1A1000818
:10A0A00029BA0008C1A10008C1A10008C1A1000887
:10A0B000C1A10008C1A10008C1A10008C1A10008F8
:10A0C000C1A10008F9B60008C1A10008C1A100089B
:10A0D000C1A10008E1B50008E9B50008F1B5000824
:10A0E000F9B50008F1A900080DAA0008C1A10008EF
:10A0F00029AA0008C1A1000845AA000861AA000811
:10A100007DAA000899AA0008C1AA0008E9AA0008C7
:10A1100011AB000839AB000861AB000889AB00083F
:10A12000B1AB0008C1A10008C1A100086DAD0008D5
:10A1300075AD0008B1B70008C1A10008C1A10008B1
:10A14000DFF810D000F09CF80048004785C00008F8
:10A15000AFF3008080D9002080F3088870470000AA
:10A16000184880474FF080404FF04021C8654000BC
:10A17000C8654010C8650846C06D40F48000C865D9
:10A1800011484FF0402148654FF04021C86D20F044
:10A190004040C8650D4880474FF00E000C494FF015
:10A1A00000000C4908800C4880470C480047FEE737
:10A1B000FEE7FEE7FEE7FEE7FEE7FEE7FEE7FEE777
:10A1C000FEE7000081B0000800100081EDAF00083C
:10A1D0000050004000600040DDB9000841A10008C7
:10A1E0002DE9F05F0546002092469B4688460646CC
:10A1F000814640241BE0284641464746224600F05F
:10A200002FF853465A46C01A914110D311461846AA
:10A21000224600F016F82D1A67EB01084F46224639
:10A220000120002100F00DF817EB00094E41201E1F
:10A23000A4F10104DFDC484631462A464346BDE826
:10A24000F09F202A04DB203A00FA02F10020704738
:10A250009140C2F1200320FA03F319439040704764
:10A26000202A04DB203A21FA02F00021704721FA6B
:10A2700002F3D040C2F120029140084319467047D2
:10A28000064C074D06E0E06840F0010394E8070043
:10A2900098471034AC42F6D3FFF756FF34C200089B
:10A2A00054C2000810B5044672B6012080F310882D
:10A2B00000BF6068074908602068FFF74DFF01F0A4
:10A2C000CDFB0A2000F048FB02480068804762B6D8
:10A2D00010BD00001400002010B503A001F0C8FB61
:10A2E00001F0DAFA10BD00007761726E696E67A343
:10A2F000BB4275734661756C742048616E646C6511
:10A30000720D0A004FF04021096A41F001014FF03F
:10A310004022116200BF4FF04021096A01F48071B0
:10A32000B1F5807FF7D14FF04021496A21F0030158
:10A330004FF0402251621146496A516200BF4FF00E
:10A340004021496A01F48071B1F5807FF7D152490B
:10A35000524A1160032806D1111F096841F080415B
:10A36000121F116007E04D49091F096821F0804163
:10A370004A4A121F11604FF4C601484A121D11606B
:10A380004FF4B20111604FF40C1111604FF45801F9
:10A3900011601160D1064FF04022D1654900D165AE
:10A3A0004910D1655101D16560B93D49096801F095
:10A3B0007F41B1F1124F37D13949096821F07F410E
:10A3C000916631E0022810D135490831096801F061
:10A3D0007F41B1F1124F27D131490831096821F08D
:10A3E0007F414FF0402291661EE003280CD12C499A
:10A3F000FC3109682B4A914216D12949F831096884
:10A400004FF0402291660FE02549091D096801F0CF
:10A410007F41B1F1124F07D12149091D096821F08F
:10A420007F414FF04022916600211C4A121D1160AD
:10A430001A49091F096821F08041184A121F11604A
:10A4400015493039121D11604FF04021096A41F061
:10A4500008014FF04022116200BF4FF04021096A0D
:10A4600001F40061B1F5006FF7D14FF04021496A66
:10A4700021F003014FF0402251621146496A41F038
:10A480000101516200BF4FF04021496A01F400719F
:10A49000B1F5007FF7D170473099D8D80438004023
:10A4A000C00020083598746770B502460B46274DEA
:10A4B0002D6845F08045254E3560351D2D78244E9C
:10A4C00045EA0604224D3035204E361D3560214DBB
:10A4D0002D6845F2AA56B5421DD14FF04025296B93
:10A4E00053B102F004051DB1114321F004010DE048
:10A4F000114381F0040109E002F004051DB191430C
:10A5000041F0040102E0914381F004014FF0402545
:10A5100029635A2010E03BB14FF040252D6B1543C5
:10A520004FF04026356306E04FF040252D6B9543F4
:10A530004FF040263563FF20044D2D1D2C602D1F4C
:10A540002D6825F08045014E356070BD0038004013
:10A550000099D8D8A400200870B504460D460720FD
:10A5600000F014FA34B1012C2AD0022C50D0032C64
:10A5700076D176E04FF04020006A40F001004FF0C5
:10A580004021086200BF4FF04020006A00F4807054
:10A59000B0F5807FF7D14FF04020406A20F00300F3
:10A5A0004FF0402148620846406A486200BF4FF0C1
:10A5B0004020406A00F48070B0F5807FF7D179E0E8
:10A5C0004FF04020006A40F008004FF04021086240
:10A5D00000BF4FF04020006A00F40060B0F5006F4B
:10A5E000F7D14FF04020406A20F003004FF04021A7
:10A5F00048620846406A40F00100486200BF4FF0E0
:10A600004020406A00F40070B0F5007FF7D151E0BF
:10A610004FF04020006A40F004004FF040210862F3
:10A6200000BF4FF04020006A00F48060B0F5806FFA
:10A63000F7D14FF04020406A20F003004FF0402156
:10A6400048620846406A40F00200486200BF4FF08E
:10A650004020406A00F48060B0F5806FF7D129E0B7
:10A6600027E04FF04020006A40F010004FF04021FA
:10A67000086200BF4FF04020006A00F48050B0F53F
:10A68000805FF7D14FF04020406A20F003004FF088
:10A69000402148620846406A40F00300486200BF1B
:10A6A0004FF04020406A00F40060B0F5006FF7D131
:10A6B00000E000BF00BF284601F025FC70BD00B5DA
:10A6C000034600F01EF84FF04020C06D40F400003B
:10A6D0004FF04021C865102B05D10846006D40F4AD
:10A6E000004008650CE04FF04020006D20F4004071
:10A6F0004FF0402108650846006D63F303000865CC
:10A7000000BD4FF04021C96D21F040404FF0402185
:10A71000C86540F080414FF04022D16540F00041D3
:10A72000D16540F04041D1657047000030B530B987
:10A73000534C646A24F47F44514D6C621AE0012842
:10A740000BD14F4C646A24F47F444D4D6C622C460F
:10A75000646A44F42A446C620CE002280AD1484C32
:10A76000646A24F47F44464D6C622C46646A44F467
:10A770007F446C6232B9424C246A24F44034404D28
:10A780002C621AE0012A0BD13D4C246A24F4403497
:10A790003B4D2C622C46246A44F400342C620CE0BD
:10A7A000022A0AD1364C246A24F44034344D2C62F7
:10A7B0002C46246A44F440342C6233B9304C646A29
:10A7C00024F47F042E4D6C621AE0012B0BD12C4C2B
:10A7D000646A24F47F042A4D6C622C46646A44F453
:10A7E0002A046C620CE0022B0AD1254C646A24F422
:10A7F0007F04234D6C622C46646A44F47F046C62CF
:10A8000031B91F4C646A24F0FF041D4D6C6222E0D4
:10A8100001290FD11B4C1A4D80352C60184C646AED
:10A8200024F0FF04164D6C622C46646A44F0AA04BE
:10A830006C6210E002290ED1124C114D80352C6053
:10A840000F4C646A24F0FF040D4D6C622C46646A60
:10A8500044F0FF046C620A4C246844F00544084D3F
:10A860002C6000BF064C246804F00044B4F1004F93
:10A87000F8D0034C246844F00104014D2C6030BD35
:10A8800000500540FFFF1F001C480068806A1B48FD
:10A890000068806C00F00F0060B118480068806CA0
:10A8A00000F00F001649086008460068134909685F
:10A8B000C1F8980011480068806A104909688867E3
:10A8C0000E480068006B0D490968C1F880000B480C
:10A8D0000068806B09490968C1F88800074800686A
:10A8E000006C06490968C1F8900004480068806C53
:10A8F00002490968C1F8980070470000C8000020AC
:10A90000D0000020024600230648824201D10123E4
:10A9100000E00023044800EB031050F82100C06958
:10A9200070470000004001408400002010B503A0E3
:10A9300001F09EF800F0B0FF10BD00007761726E6C
:10A94000696E67A3BB44656275674D6F6E20486191
:10A950006E646C65720D0A0001B581B000200A4971
:10A96000096841F27072B1FBF2F1009105E000E07C
:10A97000401C00998842FBD3002001994A1E019295
:10A980000029F4D10CBD0000AC0000200146054AAE
:10A99000106820F00F0001F00F021043014A106010
:10A9A00070470000003800400E48406800F0020088
:10A9B00040B101200C4908700A48406840F002008C
:10A9C000084948600748406C00F0020040B101208F
:10A9D000064908700348406C40F002000149486491
:10A9E0007047000000A00040D4000020D5000020E7
:10A9F00010B50021034800F0EFF80021024800F0F4
:10AA0000EBF810BD009001400040024010B501215C
:10AA1000034800F0E1F80121024800F0DDF810BD24
:10AA2000009001400040024010B50321034800F0AF
:10AA3000D3F80321024800F0CFF810BD0090014088
:10AA40000040024010B50521034800F0C5F805217B
:10AA5000024800F0C1F810BD0090014000400240E3
:10AA600010B50621034800F0B7F80621024800F0AF
:10AA7000B3F810BD009001400040024010B507211E
:10AA8000034800F0A9F80721024800F0A5F810BD1E
:10AA9000009001400040024010B50021054800F040
:10AAA0009BF80021044800F097F80021034800F0CB
:10AAB00093F810BD00A00140005002400060024029
:10AAC00010B50121054800F087F80121044800F085
:10AAD00083F80121034800F07FF810BD00A0014079
:10AAE000005002400060024010B50221054800F00D
:10AAF00073F80221044800F06FF80221034800F0C7
:10AB00006BF810BD00A00140005002400060024000
:10AB100010B50321054800F05FF80321044800F058
:10AB20005BF80321034800F057F810BD00A0014076
:10AB3000005002400060024010B50421054800F0BA
:10AB40004BF80421044800F047F80421034800F0C2
:10AB500043F810BD00A001400050024000600240D8
:10AB600010B50521054800F037F80521044800F02C
:10AB700033F80521034800F02FF810BD00A0014074
:10AB8000005002400060024010B50621054800F068
:10AB900023F80621044800F01FF80621034800F0BE
:10ABA0001BF810BD00A001400050024000600240B0
:10ABB00010B50721054800F00FF80721044800F000
:10ABC0000BF80721034800F007F810BD00A0014072
:10ABD000005002400060024070B504460D46E67920
:10ABE00031461BA000F044FF0120A840304000285F
:10ABF0002CD0E0790121A9400843E071204884422B
:10AC000004D12A4600211FA000F032FF26488442CA
:10AC100004D12A4601211BA000F02AFF23488442C8
:10AC200004D12A46022117A000F022FF20488442C6
:10AC300004D12A46032113A000F01AFF1D488442C4
:10AC400004D12A4604210FA000F012FF70BD0000BD
:10AC5000656E7465722065706F727420696E7465BC
:10AC600072727570742E63757272656E742073746F
:10AC700061747573203D20253032780D0A00000084
:10AC800000900140456E7465722045504F52542526
:10AC90006420696E746572727570742E50494E200E
:10ACA0003D2025640D0A000000A001400040024044
:10ACB00000500240006002404FF04020406A00F027
:10ACC0000302101E06D0012806D0022817D0032840
:10ACD00019D116E0114918E01148006808B9114966
:10ACE0000CE00F480068012801D10F4906E00C482C
:10ACF0000068022801D10D4900E00D4905E00D4929
:10AD000003E00D4901E0002100BF00BF4FF04020EB
:10AD10008068C0B2401CB1FBF0F0704700127A00AE
:10AD2000B400002000F36F06000E270780D1F00862
:10AD300000688909001C4E0E001BB70010B503A067
:10AD400000F096FE00F0A8FD10BD00007761726E65
:10AD5000696E67A3BB486172644661756C74204874
:10AD6000616E646C65720D0A0000000010B500F0A1
:10AD700005F810BD10B500F001F810BD08B50020B1
:10AD800000903C4800793C4908703A48C0793B49FA
:10AD900008700846007800F00100002858D13648B5
:10ADA000007800F00400042863D13348007800F0F4
:10ADB000020002281ED12F48007900F0010090B156
:10ADC0002C4840792E4909682E4A126888542D482B
:10ADD0000068401C2B4908602648807840F0080035
:10ADE0002449887045E02348807820F020002149DC
:10ADF00088703EE02048007800F0010008B31E484B
:10AE0000007800F04000402812D11F4800681F4918
:10AE10000968405C174948711C480068401C1B4980
:10AE200008601448807820F020001249887020E0E3
:10AE30001048407900909DF80000401CC0B200907E
:10AE400017E00C48807820F020000A49887010E054
:10AE50000848807900F0C000401C06498871084607
:10AE6000807940F0010088710846C07940F0010007
:10AE7000C87108BD00700140D8000020D900002032
:10AE8000E8000020DC000020E4000020E0000020BA
:10AE900030B530B9534C646A24F47F44514D6C6230
:10AEA0001AE001280BD14F4C646A24F47F444D4DC5
:10AEB0006C622C46646A44F42A446C620CE00228FA
:10AEC0000AD1484C646A24F47F44464D6C622C4697
:10AED000646A44F47F446C6232B9424C246A24F4BC
:10AEE0004034404D2C621AE0012A0BD13D4C246ABB
:10AEF00024F440343B4D2C622C46246A44F4003444
:10AF00002C620CE0022A0AD1364C246A24F4403424
:10AF1000344D2C622C46246A44F440342C6233B9FC
:10AF2000304C646A24F47F042E4D6C621AE0012BCD
:10AF30000BD12C4C646A24F47F042A4D6C622C469D
:10AF4000646A44F42A046C620CE0022B0AD1254C9A
:10AF5000646A24F47F04234D6C622C46646A44F4D2
:10AF60007F046C6231B91F4C646A24F0FF041D4DEC
:10AF70006C6222E001290FD11B4C1A4D80352C60E8
:10AF8000184C646A24F0FF04164D6C622C46646A07
:10AF900044F0AA046C6210E002290ED1124C114D4B
:10AFA00080352C600F4C646A24F0FF040D4D6C62F8
:10AFB0002C46646A44F0FF046C620A4C246844F036
:10AFC0000544084D2C6000BF064C246804F0004482
:10AFD000B4F1004FF8D0034C246844F00104014D53
:10AFE0002C6030BD00100540FFFF1F0010B5002190
:10AFF0004FF08040FFF758FA0121C807FFF754FAD5
:10B0000000214FF00040FFF74FFA10BD10B5024687
:10B01000002001B90121052A2FD2DFE802F0030C3C
:10B0200020262A004FF04023DB6923F001034FF074
:10B030004024E36122E04FF04023DB6943F0010349
:10B040004FF04024E3612346DB6823F00F03E36005
:10B050002346DB680B43E3600123A3610EE04FF05E
:10B060004023DB6803F00F0008E04FF04023D86C6A
:10B0700004E04FF04023D96400E000BF00BF10BDE2
:10B0800010B501210C20FFF70FFA10BD002100229E
:10B0900000BF11E00846002208E000F001031BB1E8
:10B0A000074B83EA500000E04008521C082AF4D302
:10B0B000044B43F82100491CFF29EBD970470000DD
:10B0C0002083B8EDF000002010B503A000F0D0FC04
:10B0D00000F0E2FB10BD00007761726E696E67A33D
:10B0E000BB4D656D4D616E6167652048616E646C36
:10B0F00065720D0A0000000010B503A000F0B8FC56
:10B1000000F0CAFB10BD00007761726E696E67A324
:10B11000BB4E4D492048616E646C65720D0A00009B
:10B120002DE9F0410746884614461D46284600F0A2
:10B1300033F8C5F1030007FA00F60720284100EABA
:10B140000800064306F00706E21704EBD26252112C
:10B15000920002F1E022D2F800212146E31704EB2D
:10B16000D3635B11A4EB431C012303FA0CF31A43D2
:10B170002046E31704EBD3635B119B0003F1E0234C
:10B18000C3F800210348005D40EA46100149085514
:10B19000BDE8F08100E400E00146072323EA010254
:10B1A0001202054B18684FF6FF031840034B184373
:10B1B0001043014B186070470CED00E00000FA05E9
:10B1C0004A0A52020243014B1A60704708ED00E040
:10B1D00010B57348446C04F0010040B171A000F058
:10B1E00047FC6F48406C40F001006D49486404F032
:10B1F0000200022808D170A000F03AFC6848406CB8
:10B2000040F002006649486404F01000102808D19C
:10B210006EA000F02DFC6248406C40F010006049C8
:10B22000486404F02000202808D16DA000F020FC24
:10B230005B48406C40F020005949486404F4807039
:10B24000B0F5807F13D15648806800F48010B0F5C7
:10B25000801F03D167A000F00BFC02E06BA000F0A0
:10B2600007FC4F48406C40F480704D49486404F43A
:10B270000070B0F5007F08D16AA000F0F9FB4848E3
:10B28000406C40F400704649486404F48060B0F5B6
:10B29000806F13D14248806800F40010B0F5001FA1
:10B2A00003D166A000F0E4FB02E06AA000F0E0FB3E
:10B2B0003B48406C40F480603949486404F40060C5
:10B2C000B0F5006F08D169A000F0D2FB3448406CA3
:10B2D00040F400603249486404F48050B0F5805F67
:10B2E00013D12F48806800F48000B0F5800F03D19F
:10B2F00064A000F0BDFB02E068A000F0B9FB2848A4
:10B30000406C40F480502649486404F40050B0F585
:10B31000005F08D167A000F0ABFB2148406C40F40F
:10B3200000501F49486404F48040B0F5804F13D1A9
:10B330001B48806800F40000B0F5000F03D163A043
:10B3400000F096FB02E067A000F092FB1448406C0E
:10B3500040F480401249486404F40040B0F5004FC6
:10B3600008D166A000F084FB0D48406C40F400401A
:10B370000B49486404F48030B0F5803F08D165A0E3
:10B3800000F076FB0648406C40F480300449486485
:10B390000348006A634908430149086210BD000080
:10B3A000004003405043492056445F4C20746F7561
:10B3B0006368210D0A0000005043492056445F484D
:10B3C00020746F756368210D0A0000005043492006
:10B3D00054445F4C20746F756368210D0A000000AF
:10B3E0005043492054445F4820746F756368210DB1
:10B3F0000A0000005344494F2064796E616D69630F
:10B400002D3020746F756368210D0A005344494F35
:10B41000207374617469632D3020746F75636821C3
:10B420000D0A00005344494F207374617469632D01
:10B430003120746F756368210D0A00005344494F31
:10B440002064796E616D69632D3120746F75636856
:10B45000210D0A005344494F207374617469632DB0
:10B460003220746F756368210D0A00005344494F00
:10B47000207374617469632D3320746F7563682160
:10B480000D0A00005344494F2064796E616D696371
:10B490002D3220746F756368210D0A005344494FA3
:10B4A000207374617469632D3420746F756368212F
:10B4B0000D0A00005344494F207374617469632D71
:10B4C0003520746F756368210D0A00005344494F9D
:10B4D0002064796E616D69632D3320746F756368C4
:10B4E000210D0A005344494F207374617469632D20
:10B4F0003620746F756368210D0A00005344494F6C
:10B50000207374617469632D3720746F75636821CB
:10B510000D0A00006E7672616D20636C65616E21AC
:10B520000D0A000000FFFF000448006840F01F0003
:10B530004FF04021C1F8900070470000904000405B
:10B540001349098821F00101114A11801146098827
:10B5500041F00401118001210E4A11800E4A117040
:10B560000E4909780E4A1170114609786C290DD0E0
:10B57000012004E00949095C094A1154401C0949A9
:10B5800009888842F6DB0021064A118070470000D6
:10B590000070004032000020340000200005002030
:10B5A000003B0020300000200A48008840F00400E2
:10B5B0000849088008480078401C07490870084678
:10B5C0000078052804DB002008700120034908707A
:10B5D00070470000008000407600002074000020CA
:10B5E00000B500F00DF800BD00B500F009F800BD91
:10B5F00000B500F005F800BD00B500F001F800BD91
:10B6000000201F4908781E496C3991F8441001F058
:10B61000100141B11A492839097841F01001184A3E
:10B620006C3A82F8441016492639097801F0100165
:10B6300039B113492639097841F0100210492639E9
:10B640000A700F492439097801F0100141B10C4901
:10B650002439097841F01001094A6C3A82F84810FF
:10B6600007492239097801F0100139B1044922391A
:10B67000097841F01002024922390A70704700002F
:10B680006C80014010B503A000F0F2F900F004F95D
:10B6900010BD00007761726E696E67A3BB50656E66
:10B6A0006453562048616E646C65720D0A00000098
:10B6B0002DE9F04104460D4617460026E000B0FB98
:10B6C000F5F0401CC0F345000A498872A000B0FBA9
:10B6D000F5F08609300A48700E700846807840F010
:10B6E0003C0088700223202200210846FFF718FD45
:10B6F000BDE8F081003001400648407905484079B6
:10B7000000F01000102803D102498879487900BF61
:10B71000704700000040014070B504460D46002609
:10B7200002233D2200210846FFF7FAFCE000B0FBAF
:10B73000F5F0401CC0F345001B498872A000B0FB27
:10B74000F5F08609300A48700E700846C07820F07F
:10B750001000C8700846C07820F00200C870402071
:10B760008874002088730846807B40F084008873CA
:10B770000846C07C40F00500C8740846C07840F018
:10B780000400C8700846807840F01C0088700846A5
:10B79000007C40F0010008748B15044A0221024825
:10B7A00000F0CCFB70BD000000D00140406F0020D5
:10B7B00070B5214C607900F0100000283BD004E007
:10B7C000607C00F0120000B104E0607C00F0010039
:10B7D0000028F5D000BFA579E07C40F00100E074BE
:10B7E00002212046FFF78EF81449088001201449F1
:10B7F00008701248018813A000F03AF91448006854
:10B800000E4909880844124908604FF48073114AB0
:10B810000221204600F092FB01200F4908700F48DA
:10B820008679467905480088FF2804DC08480168C5
:10B830000BA000F01DF970BD00D001407C0000207D
:10B84000447900206C656E3A25640D0A0000000002
:10B8500024000020406F0020010000200030014043
:10B860006E756D626572313D25640D0A0000000041
:10B8700010B503A000F0FCF800F00EF810BD0000B9
:10B880007761726E696E67A3BB5356432048616E41
:10B89000646C65720D0A000010B5FEF732FF4FF0C0
:10B8A0004020C06D40F008004FF04021C86510BD39
:10B8B000704700002DE9FF4704460D4617464FF03C
:10B8C0000009344B0FCB8DE80F00C8460026032C2F
:10B8D00001DC002C10DAFFF7EFF92F490860002196
:10B8E0000220FFF793FB401C2B490968B1FBF0F0E5
:10B8F0002A490860BDE8FF87FFF7DEF9804628483F
:10B900000460032C01D105B901255DF82410681CE1
:10B91000B1FBF0F62348864205D146450ED0032000
:10B92000FEF7CDFE0AE02048804505D8864203D9BF
:10B930000120FEF7C4FE01E04FF001092046FEF7AA
:10B94000E1FC29460120FEF707FE39460120FFF7FA
:10B950005DFBFFF7B1F91049086000210220FFF7F5
:10B9600055FB401C0C490968B1FBF0F00B4908601D
:10B97000094800680C49884203D81020FEF79FFE52
:10B9800005E0B9F1000F02D00120FEF798FE00BFDC
:10B99000B0E7000024C20008AC000020B000002086
:10B9A000B400002080D1F0080087930310B50A4846
:10B9B00000F0BBFA012200210220FFF77BFF0023E9
:10B9C0001A4601211846FEF7B1FE00231A4601214E
:10B9D0001846FFF75DFA10BD90D0030006480068D6
:10B9E00040F470000449086004486FF308000249FD
:10B9F000803908607047000088ED00E000A0000872
:10BA000000B500F001F800BD0648008840F00800CD
:10BA10000449088000BF0348008800F08000002827
:10BA2000F9D17047006000407047000010B503A0D6
:10BA300000F01EF8FFF730FF10BD00007761726E56
:10BA4000696E67A3BB55736167654661756C742049
:10BA500048616E646C65720D0A00000045F2555035
:10BA60000249C8804000C880704700000050004074
:10BA70000FB4054B10B503A9044A029800F018F85A
:10BA800010BC5DF814FB000069C00008EC00002049
:10BA900002E008C8121F08C1002AFAD17047704797
:10BAA000002001E001C1121F002AFBD170470000F5
:10BAB0002DE9FF4F8DB00F460546002606E02528EC
:10BAC0000BD0DDE90F1290476D1C761C28780028FA
:10BAD000F5D111B03046BDE8F08F0024A246A14652
:10BAE0000122E94900E0044315F8013F203B02FA36
:10BAF00003F00842F7D128782A2810D06FF02F02DF
:10BB00002878A0F13001092914D80AEB8A0102EB48
:10BB1000410144F0020400EB010A6D1CF0E701CF83
:10BB20005FEA000A03D544F40054CAF1000A44F065
:10BB300002046D1C28782E2817D115F8010F44F047
:10BB400004042A280ED06FF02F022878A0F13001CB
:10BB500009290AD809EB890102EB410100EB01092F
:10BB60006D1CF2E757F8049B6D1C28786C280FD0E9
:10BB700006DC4C2817D068280DD06A2814D104E0C0
:10BB8000742810D07A280FD10DE044F400140AE094
:10BB900044F4801401E044F440146978814202D1F5
:10BBA00004F580146D1C6D1C28786E281ED00CDCEA
:10BBB000632830D004DC00288BD0582811D19FE0B6
:10BBC000642867D069280CD164E073282DD004DC88
:10BBD0006F2872D0702804D194E075286ED0782830
:10BBE0006DD0DDE90F129047761C4BE1C4F3025093
:10BBF000022806D0032809D0042801CF09D0066006
:10BC000040E101CFF117C0E900613BE101CF0680BF
:10BC100038E1067036E117F8040B8DF800000020BB
:10BC20008DF80100EB46012003E057F804BB4FF00C
:10BC3000FF3061074FF0000102D40DE008F101016F
:10BC4000884649450FDA8045F8DB1BF808100029C3
:10BC5000F4D108E008F1010188468142FADB1BF8C3
:10BC600008100029F6D1DDE90F23AAEB0800814670
:10BC7000214600F031F9304400EB080604E0DDE92C
:10BC80000F121BF8010B9047B8F10108F7D22146BB
:10BC90004846F2E00A21C4F302524FF0000B08912B
:10BCA000022A04D001CFC117032A09D00AE0FF1DE0
:10BCB00027F00707F7E8020108E02CE01EE01FE08C
:10BCC00000B2C117042A01D140B2C117021E71F19E
:10BCD000000206DA0023D0EB030063EB01012D2202
:10BCE00002E0220504D52B228DF82420012203E056
:10BCF000E20701D02022F7E7904653E00A210BE04B
:10BD0000102109E010214FF0000B44F004044FF023
:10BD10000809089103E008214FF0000B0891C4F3D3
:10BD20000252022A04D001CF0021032A06D006E0E5
:10BD3000FF1D27F00707F7E8020103E080B2042A9D
:10BD400000D1C0B24FF0000822072BD52A78702A04
:10BD500007D0DDF820C08CF0100C5CEA0B0C05D08D
:10BD60000EE040228DF82420012208E050EA010371
:10BD700006D030238DF824308DF8252002229046FD
:10BD8000089B83F0080353EA0B030BD150EA01022E
:10BD900001D1620706D530228DF824204FF001082A
:10BDA000A9F101092A78582A04D038A20B9208AACE
:10BDB0000A920BE03AA2F9E75B46089AFEF710FAFE
:10BDC0000B9B9B5C0A9A521E0A92137050EA010266
:10BDD000F2D10A98ADEB000000F1200B600702D50C
:10BDE00024F4803401E04FF00109D94502DDA9EBCC
:10BDF0000B0000E0002000EB0B0141440890AAEB8F
:10BE0000010AE00306D4DDE90F232146504600F085
:10BE100063F806444FF0000908E009A911F8090089
:10BE2000DDE90F12904709F10109761CC145F4DBE9
:10BE3000E0030CD5DDE90F232146504600F04CF815
:10BE4000064404E0DDE90F1230209047761C089983
:10BE5000481E08900029F5DC08E00A980A99007845
:10BE6000491C0A91DDE90F129047761CBBF10001D5
:10BE7000ABF1010BF1DC21465046DDE90F2300F068
:10BE800019F806446D1C21E60928010030313233CF
:10BE90003435363738396162636465660000000006
:10BEA00030313233343536373839414243444546F0
:10BEB000000000002DE9F041044600251E4617460B
:10BEC000880404D405E039462020B0476D1C641E68
:10BED000F9D52846BDE8F0812DE9F041044600255A
:10BEE0001E469046C80301D5302700E0202788046D
:10BEF00004D505E041463846B0476D1C641EF9D5AF
:10BF00002846BDE8F0814FF04021896821F0FF010B
:10BF10004FF04022916011468968014391601146BB
:10BF2000896941F002019161704701B500BF009835
:10BF3000411E00910028FAD108BD0000F0B5054669
:10BF40000C46002100200026424FBD4201D10121B4
:10BF500000E000210127A74047EA072C3E4F57F891
:10BF60002170D7F8E07027EA0C07DFF8ECC05CF826
:10BF700021C0CCF8E0700027DFF8DCC05CF821C0FD
:10BF8000CCF8D870AF1DDFF8D4C00CEB011C5CF806
:10BF900024C0CCF80070314F07EB011757F824701C
:10BFA000BA602F4FDFF8B4C00CEB011C5CF824C062
:10BFB000CCF81870294F07EB011757F82470FB6174
:10BFC0000127DFF894C05CF821C0CCF8D8704FF49A
:10BFD000C867DFF888C00CEB011C5CF824C0CCF803
:10BFE0004070204FBD420AD14FF4B067DFF86CC0FB
:10BFF0000CEB011C5CF824C0CCF8447016E0154F23
:10C00000BD4209D10027DFF854C00CEB011C5CF8DD
:10C0100024C0CCF8447009E04FF4D067DFF83CC08E
:10C020000CEB011C5CF824C0CCF844700127A7403D
:10C0300047EA0727DFF820C05CF821C0DCF8E0C041
:10C0400047EA0C07DFF810C05CF821C0CCF8E070BC
:10C05000F0BD000000400140A4000020840000204A
:10C060000004200000300140024600BF044840792F
:10C0700000F040000028F9D0D0B2014B9871704711
:10C080000030014000214A48FFF79AF8FFF78EFC84
:10C0900062B600224FF4612146480068FFF708FBB2
:10C0A000454846490860FEF7F1FF434843490860A8
:10C0B00043A0FFF7DDFC4FF461213E480068FFF725
:10C0C0002BFB00BF72E0FFF7C9FC43480078012852
:10C0D0006CD1FFF7C3FC41480078A52820D13F4828
:10C0E00040785A281CD13D488078082818D13B4810
:10C0F000C078012814D13948007988B93748407987
:10C1000070B936488079FF280AD13448C079FE28B2
:10C1100006D133A0FFF7ACFC2748FEF7C3F824E0B4
:10C120002E480078A52820D12C4840785A281CD1C8
:10C130002A488078082818D12848C078042814D1C3
:10C1400026480079902810D12448407968B92348BE
:10C150008079FF2809D12148C079FE2805D125A082
:10C16000FFF786FC2848FEF79DF828480068284914
:10C170000988084425490860002406E01748015D45
:10C1800024A0FFF775FC601C84B22148008884421B
:10C19000F4DB1CA0FFF76CFC00201D4908800E4951
:10C1A00008701A4801681CA0FFF762FC8BE70000CA
:10C1B00000A00008B0000020000001080C000020D2
:10C1C0002A2A2A626F6F746C6F6164657231212153
:10C1D0002A2A0D0A0000000001000020406F002004
:10C1E000656E746572204150505F41444452210D88
:10C1F0000A000000656E74657220415050325F4144
:10C20000444452210D0A0000009004082800002038
:10C210007C000020202578006E756D6265723D25DA
:10C22000640D0A0000F36F06000E270780D1F008A6
:10C230000068890954C2000800000020F0000000D6
:10C2400090BA000844C30008F000002090D8000015
:10C25000A0BA00080000000000000000000000007C
:10C2600000000000000000000000000000000000CE
:10C2700000000000000000000000000000000000BE
:10C2800000000000000000000000000000000000AE
:10C29000000000000000000000000000000000009E
:10C2A000000000000000000000000000000000008E
:10C2B000000000000000000000000000000000007E
:10C2C000000000000000000000000000000000006E
:10C2D00000000000000000000060044058600440BE
:10C2E000B06004400861044000700440587004408D
:10C2F000B070044008710440C0620440C072044041
:10C300000000000000000000030000000060044086
:10C3100058600440B060044008610440C0620440BA
:10C3200000000000000000000000000000FF00000E
:10C3300000000000000000000000000000000000FD
:04C3400000000000F9
:040000050800A1410D
:00000001FF
